:020000040800F2
:1000000000040020A1020008A3020008A3020008C7
:10001000A3020008A3020008A3020008A30200082C
:10002000A3020008A3020008A30200089127000809
:10003000A3020008A3020008A3020008A30200080C
:10004000A3020008A3020008A3020008A3020008FC
:10005000A3020008A3020008D53C0008013D0008E7
:100060002D3D0008593D0008853D0008A302000809
:10007000A3020008A3020008A3020008A3020008CC
:10008000A3020008A3020008A3020008A3020008BC
:10009000A3020008A3020008A3020008B13D000863
:1000A000A3020008A3020008A3020008A30200089C
:1000B000A3020008A3020008A3020008A30200088C
:1000C000A3020008A3020008A3020008A30200087C
:1000D000A3020008A3020008A3020008A30200086C
:1000E000193E0008A3020008A3020008A3020008AA
:1000F000A3020008A3020008A3020008A30200084C
:10010000A3020008A302000855390008A302000852
:10011000A3020008A3020008A3020008A30200082B
:10012000A3020008A3020008A3020008A30200081B
:10013000A3020008A3020008A3020008A30200080B
:10014000A3020008A3020008A3020008A3020008FB
:10015000A3020008A3020008A3020008A3020008EB
:10016000A3020008A3020008A3020008A3020008DB
:10017000A3020008C9320008A3020008A302000875
:10018000A3020008A302000825100008A30200082B
:10019000A3020008A3020008A3020008A3020008AB
:1001A000A3020008A3020008A3020008A30200089B
:1001B000A3020008A3020008A3020008A30200088B
:1001C000A3020008A3020008A3020008A30200087B
:1001D000A3020008B5320008A3020008A302000829
:1001E000A3020008A3020008A3020008A30200085B
:1001F000A3020008A3020008A3020008A30200084B
:10020000A3020008A3020008A3020008A30200083A
:10021000A3020008A3020008A3020008A30200082A
:10022000A3020008A3020008A3020008A30200081A
:10023000A3020008A3020008A3020008A30200080A
:10024000A3020008A3020008A3020008A3020008FA
:10025000A3020008A3020008A3020008A3020008EA
:10026000A3020008A3020008A3020008A3020008DA
:10027000A3020008A3020008A3020008A3020008CA
:10028000A3020008A3020008A3020008A3020008BA
:10029000A3020008A3020008A3020008A3020008AA
:1002A00002E000F000F8FEE772B6394880F30888F3
:1002B000384880F3098838484EF60851CEF20001DC
:1002C000086040F20000CCF200004EF63471CEF22D
:1002D00000010860BFF34F8FBFF36F8F40F2000043
:1002E000C0F2F0004EF68851CEF200010860BFF374
:1002F0004F8FBFF36F8F4FF00000E1EE100A4EF604
:100300003C71CEF200010860062080F31488BFF330
:100310006F8F02F07BFA03F09BFA4FF055301F49C4
:100320001B4A91423CBF41F8040BFAE71C49194AA9
:1003300091423CBF41F8040BFAE71A491A4A1B4B99
:100340009A423EBF51F8040B42F8040BF8E7002034
:100350001749184A91423CBF41F8040BFAE702F0F2
:1003600099FA03F0E9FA144C144DAC4203DA54F84C
:10037000041B8847F9E700F03FF8114C114DAC42DF
:1003800003DA54F8041B8847F9E702F081BA000049
:1003900000040020002400200000000800000020CD
:1003A00000040020784200080024002038240020A7
:1003B0003824002050390020A0020008A0020008C4
:1003C000A0020008A00200082DE9F04F2DED108AD0
:1003D000C1F80CD0D0F80CD0BDEC108ABDE8F08F7D
:1003E000002383F311882846A047002001F040FE37
:1003F00001F0F0FD00DFFEE738B5204C6FF074032C
:10040000002523701E236570A570E5702571657148
:10041000A571E57125726572A372E57200F02AFD7F
:1004200020B10E2325726572A372E57202F088F97D
:10043000044602F0A7F90546D8B9114B9C421AD0E0
:1004400001339C4218BF054641F2883404BF0125A0
:100450000024002002F07EF90DB100F0B7F800F0A2
:1004600073FD00F08BFC204600F070F900F0AEF850
:10047000F9E70024EDE70446EBE700BF382400204D
:10048000010007B008B500F0F7FBA0F120035842C7
:10049000584108BD07B5054B02211B88ADF8043053
:1004A00001A800F055FC03B05DF804FB383F0008DC
:1004B000064991F8243033B100230822086A81F8F4
:1004C000243000F07FBC0120704700BF582400207A
:1004D0002DE9F84F234C94F82430054688461746FA
:1004E0008BBB2E46DFF87C90002F38D094F824A0E8
:1004F000BAF1000F05D12022FF214846266200F004
:1005000011FDCAF10805BD4228BF3D465FFA85FBD3
:10051000AD0041462A4604EB8A0000F0D9FC94F86D
:100520002430A7EB0B079B445FFA8BFBBBF1080F52
:100530002E44A844FFB284F824B0D5D1FFF7B8FF09
:100540000028D1D108E0266A06EB8306B042C9D064
:10055000FFF7AEFF0028C4D10020BDE8F88F0120CE
:10056000BDE8F88F5824002010B5202383F31188AC
:100570001248C3680BB101F001FE0023104A0F4876
:100580004FF47A7101F0BEFD002383F311880D4C06
:10059000236813B12368013B2360636813B1636868
:1005A000013B6360084B1B7833B9636823B90220B1
:1005B00000F07CFC3223636010BD00BF44240020A7
:1005C0006905000888290020802400202DE9F041D9
:1005D000544B554953F8042F013201D1BDE8F08145
:1005E0008B42F7D1514C524B22689A4240F298808C
:1005F000504B9B6803F1006303F500339A4280F08F
:100600008F80002000F0D6FB4B4B0220187000F0CA
:1006100041FC4A4BD3F8E8200022C3F8E820D3F885
:100620001011C3F81021D3F81011D3F8EC10C3F84F
:10063000EC20D3F81411C3F81421D3F81411D3F813
:10064000F010C3F8F020D3F81811C3F81821D3F82C
:100650001811D3F8801041F00061C3F88010D3F86E
:10066000801021F00061C3F88010D3F88010D3F817
:10067000801041F00071C3F88010D3F8801021F091
:100680000071C3F88010D3F8803072B62C492D4B1E
:100690000B601D682468BFF34F8FBFF36F8F2A4B29
:1006A000C3F88420BFF34F8F5A6922F480325A6115
:1006B000BFF34F8FD3F88020C2F3C906C2F34E3286
:1006C0005201B70743F6E07E02EA0E08384631468B
:1006D000013948EA000CB1F1FF3FC3F874C200F1E0
:1006E0004040F5D1203A12F1200FEDD1BFF34F8FEA
:1006F000BFF36F8FBFF34F8FBFF36F8F5A6922F431
:1007000000325A610022C3F85022BFF34F8FBFF36B
:100710006F8F202383F31188AD4685F30888204727
:10072000BDE8F081FCFF01081C000208040002087B
:10073000FFFF0108382400208024002000440258D4
:1007400008ED00E00000020800ED00E02DE9F04FA8
:10075000B04C97B020228146FF210EA8A66800F079
:10076000E1FBAD4A1378A346A3B9AC480121C360AD
:100770001170202383F31188C3680BB101F0FEFCD4
:100780000023A74AA5484FF47A7101F0BBFC00236F
:1007900083F31188B9F1000F02D0A24BC3F8009087
:1007A000A14BA04A00241C70546025462746984659
:1007B000012000F06FFBB9F1000F00F02282994B8D
:1007C0001B68002B40F01D8217B0BDE8F08F02209F
:1007D000FFF758FE002840F00E82944B1B88ADF8BE
:1007E0002430022109A800F0B3FAE1E74FF47A704F
:1007F00000F042FA031E0193EFDB0220FFF742FEF6
:1008000082460028E9D0019B581E042800F2F58199
:10081000DFE800F0030D1013160016A8052340F8BA
:10082000343D042100F094FA5446002752E004219C
:100830007848F7E704217E48F4E704217D48F1E792
:100840001C24204600F0B8FA04340990042109A8B9
:1008500000F07EFA2C2CF4D1E6E7002DBDD0002C60
:10086000BBD00220FFF70EFE0546002800F0C7812E
:10087000012000F09FFA022088F8000000F00AFB37
:100880000024E3B21846019300F0A4FA824648B16E
:10089000019B184600F0AEFA01340028F1D12C4635
:1008A000654B9BE70123022088F8003000F0E4FA52
:1008B0005646DBF808309E4206D2304600F07CFAFD
:1008C0000130ECD10436F4E7564B002688F800607E
:1008D0005E602C4600F02EFB1DB1002C18BF4FF0BF
:1008E0000009FFF7D7FD63E7002D3FF476AF002C3A
:1008F0003FF473AF022088F8000000F0CBFA3220FA
:1009000000F0BAF9B0F1000AC0F279811AF00305DB
:1009100040F07581DBF8082006EB0A03934200F2F1
:100920006E81BAF5807F00F26A81444B0193554590
:100930000DDA4FF47A7000F09FF90290029A002AC3
:10094000C0F25D81019B029AEA540135EEE7C820AE
:10095000FFF798FD0546002800F051811F2E11D8A1
:10096000C6F12004544528BF54460EAB26F00300C0
:1009700022463249184400F0ABFA2246FF212F48A4
:1009800000F0D0FA4FEAAA0A5FFA8AF22B49304601
:10099000FFF79EFD0446002881D006EB8A06054637
:1009A00098E70220FFF76EFD00283FF416AFFFF72F
:1009B0007FFD00283FF411AF00229246DBF808309B
:1009C0009A4259D21F2A1ED80E9B01331BD022F007
:1009D000030316A90B4453F8203C099318484368B5
:1009E00083B3174800210DF1240E11F80E3083EA6D
:1009F0000A03DBB2013150F82330042983EA1A2AB2
:100A0000F3D10432DAE71046019200F0D5F9019AE9
:100A10000990E3E7382400208425002044240020A6
:100A20006905000888290020802400203A3F00083A
:100A30003C240020402400203C3F00088424002067
:100A40008825002019464FF0080E11F0010F4FEADB
:100A500051011FBF81F06D4181F4380181F40341E0
:100A600081F02001BEF1010EEFD140F823100133D7
:100A7000B3F5807FE6D1B4E716A8042140F84CAD69
:100A800000F066F926E716A8002340F8343D6421FB
:100A900000F02AF900287FF4A0AE0220FFF7F2FC54
:100AA00000283FF49AAE099800F0B6F916AB43F867
:100AB000480D04211846E3E716A8002340F8343D0A
:100AC000642100F011F900287FF487AE0220FFF7BF
:100AD000D9FC00283FF481AE099800F09FF916ABCD
:100AE00043F8440DE5E70220FFF7CCFC00283FF473
:100AF00074AE00F099F916AB43F8400DD9E7022027
:100B0000FFF7C0FC00283FF468AE09A9142000F0EC
:100B100091F9824616A8042140F83CAD00F018F97E
:100B2000514609A8ACE7322000F0A6F8B0F1000A5F
:100B3000FFF653AE1AF0030F7FF44FAEDBF8082038
:100B40000AEB070393423FF648AE0220FFF79AFCF8
:100B500000283FF442AE2AF0030ABA44BA453FF4F3
:100B6000B9AE384600F028F90421089008A800F032
:100B7000EFF80437F2E74FF47A70FFF783FC0028B0
:100B80003FF42BAEFFF794FC00283FF489AE0E9B98
:100B900001330CD008220EA90020FFF799FC002891
:100BA0003FF47EAE2022FF210EA800F0BBF9FFF734
:100BB00071FC304801F062FA06E616A8002340F8FE
:100BC000343D642100F090F8824600287FF405AEA1
:100BD0000220FFF757FC00283FF4FFADFFF75AFC57
:100BE00041F2883001F04AFA099800F0E7F9D1465D
:100BF00000F0A0F9DCE505466CE60027EDE52546AA
:100C0000EBE5002000F038F80290029B002BFFF685
:100C1000D2AD012000F030F9029B213B122B3FF6B0
:100C2000C7AD01A252F823F0CF070008ED07000876
:100C30005B080008B1070008B1070008B107000809
:100C4000E9080008270B0008A3090008870A000824
:100C5000B90A0008E70A0008B1070008FF0A0008FF
:100C6000B1070008770B0008D5080008B107000895
:100C7000BB0B0008A08601002DE9F34702AE00245B
:100C80004FF47A7506F8014D144FDFF8588045434C
:100C900097F900305A1C5FFA84F901D0A34212D1AF
:100CA00058F8240003680122D3F820A031462B46CF
:100CB000D047012807D10A4B9DF8070083F8009020
:100CC00002B0BDE8F0870134022CE1D14FF4FA7094
:100CD00001F0D4F94FF0FF30F2E700BF002400200C
:100CE000AC290020403F00082DE9F0474FF47A7509
:100CF000144FDFF8588006464D43002497F9003022
:100D00005A1C5FFA84F901D0A34210D158F824008C
:100D100003680422D3F820A031462B46D04704288C
:100D200005D1094B83F800900020BDE8F08701341D
:100D3000022CE3D14FF4FA7001F0A0F94FF0FF302C
:100D4000BDE8F08700240020AC290020403F0008C7
:100D500030B4074B1A78074B53F822402368DD69FB
:100D6000054B0A46AC460146204630BC604700BFF2
:100D7000AC290020403F0008A0860100F8B501F032
:100D8000C3FB094C094E0A4F2070002530682378B8
:100D9000834207D901F0B4FB336805440133BD42F7
:100DA0003360F3D9F8BD00BFAD29002090290020A1
:100DB000FFFF010001F078BC00F1006000F5003099
:100DC0000068704700F10060920000F5003001F00B
:100DD00005BC0000054B1A68054B1B789B1A834223
:100DE00002D9104401F08CBB0020704790290020EC
:100DF000AD29002038B5074D04462868204401F08D
:100E000085FB28B928682044BDE8384001F090BB34
:100E100038BD00BF9029002000207047014BC0580A
:100E2000704700BF00E8F11F014B1868704700BF12
:100E30000010005C70B50E4B5C6893F908600138D7
:100E40000A18013C0B4693420FD214F9015F581C5B
:100E50001DB1034600F8015CF5E72C2482421C70AA
:100E600001D9981C5E70401A70BD1846FBE700BFA0
:100E70000424002000207047022804D14FF400020F
:100E8000034B9A6170470128FCD14FF48002F7E7C9
:100E900000080258022803D18022034B9A61704750
:100EA0000128FCD14022F8E700080258022805D1A9
:100EB000064A536983F08003536170470128FCD1CF
:100EC000024A536983F04003F6E700BF0008025866
:100ED00010B50023934203D0CC5CC4540133F9E72E
:100EE00010BD000030B5441E14F9010F0B4660B16F
:100EF00093F90050854201F1010106D11AB993F925
:100F00000020801A30BD013AEEE7002AF7D11046E2
:100F100030BD000002460346981A13F9011B002950
:100F2000FAD1704702440346934202D003F8011BF2
:100F3000FAE77047024B1A78024B1A70704700BFED
:100F4000AC2900200024002038B5164C164D204650
:100F500000F0C6FB2946204600F0EEFB2D68134842
:100F6000D5F89020D2F8043843F00203C2F80438D0
:100F700001F084F80E49284600F0EEFCD5F89020E8
:100F80000C48D2F804380C4923F00203C2F80438A4
:100F9000A0424FF4E1330B6003D0BDE8384000F0CD
:100FA000FDBA38BD5C2E00201440000840420F00FE
:100FB0003C400008B02900209429002038B50B4B94
:100FC0001A780B4B53F822400A4B9C4205460CD032
:100FD000094B002118461822FFF7A4FF05600146BF
:100FE0002046BDE8384000F0D9BA38BDAC29002011
:100FF000403F00085C2E002094290020024A13681C
:1010000043F0C0031360704700780040044B5A68F7
:1010100010439A6858600AB1181D1047704700BF06
:10102000B02900202DE9F84F404EF56D2F68EC698E
:101030002C62210718D014F0080F0CBF002080206C
:10104000E20748BF40F02000A30748BF40F040003F
:10105000610748BF40F48070202383F31188FFF7B5
:10106000D5FF002383F31188E20509D5202383F3FC
:1010700011884FF40070FFF7C9FF002383F3118834
:10108000DFF8A8A04FF020094FF0000B14F0200863
:1010900032D13B0615D5DFF898A04FF02009200685
:1010A0000FD589F31188504600F0ECF9002830DAAA
:1010B0000820FFF7ABFF27F080032B60002383F3AA
:1010C000118879060DD562060BD5202383F311888C
:1010D000F26C336D9A4201D1336C03BB002383F36E
:1010E0001188E30604D5B26E13690BB150699847B5
:1010F000BDE8F84F01F05CBB89F31188AB8C96F822
:1011000064105046194000F057FA8BF31188EC69CF
:10111000BCE780B2288588F31188EC69BFE710200E
:1011200027F04007FFF772FF2F60D7E7B0290020B4
:10113000E829002013B5104C204600F023FA04F1F2
:101140001400009400234FF400720C4900F0E4F8FE
:1011500004F1380000940A4B0A494FF4007200F081
:101160005DF9094BE365094B23660C21522002B05F
:10117000BDE8104000F05EB8B02900201C2A002015
:10118000FD0F00081C2C00200078004000E1F50550
:10119000254B002908BF1946037C8166012B30B519
:1011A00011D1224B98420ED1214BD3F8E82042F0C6
:1011B0008042C3F8E820D3F8102142F08042C3F8FF
:1011C0001021D3F810310A68036EC46D03EB52038B
:1011D000B3FBF2F34A68150442BF23F0070503F09E
:1011E000070343EA4503E3608B6843F04003636011
:1011F000CB6843F00103A36042F4967343F001030C
:10120000236051054FF0FF33236205D512F0102201
:1012100005D0B2F1805F04D080F8643030BD7F2308
:10122000FAE73F23F8E700BF583F0008B029002045
:101230000044025800F1604300F01F02400903F52A
:10124000614309018000C9B200F1604083F80013D6
:1012500000F5614001239340C0F88031036070477E
:10126000F8B5154682680669AA420B46816938BFFF
:101270008568761AB542044607D218462A46FFF713
:1012800027FEA3692B44A3610DE011D9324618460D
:10129000FFF71EFEAF1B3A46E1683044FFF718FE29
:1012A000E2683A44A261A3685B1BA3602846F8BDCC
:1012B00018462A46FFF70CFEE368E4E783682DE949
:1012C000F041044693421546266938BF8568406957
:1012D000361AB5420F4606D22A46FFF7F9FD636972
:1012E0002B4463610DE012D93246A5EB0608FFF7E7
:1012F000EFFD4246B919E068FFF7EAFDE2684244B3
:101300006261A3685B1BA3602846BDE8F0812A46A2
:10131000FFF7DEFDE368E4E710B50A440024C3618B
:10132000029B006040608460C16081614161026134
:10133000036210BD08B582694369934201D1826896
:1013400082B98268013282605A1C42611970426916
:1013500003699A4201D3C3684361002100F0AAFEE9
:10136000002008BD4FF0FF3008BD000070B52023FD
:1013700004460E4683F31188A568A5B1A368A26947
:10138000013BA360531CA36115782269934224BFDB
:10139000E368A361E3690BB120469847002383F318
:1013A0001188284670BD3146204600F073FE0028A3
:1013B000E2DA85F3118870BD2DE9F74F05460F4637
:1013C00090469A46D0F81C90202686F311884FF05C
:1013D000000B144664B1224639462846FFF740FF09
:1013E000034668B95146284600F054FE0028F1D063
:1013F000002383F31188A8EB040003B0BDE8F08F4D
:10140000B9F1000F03D001902846C847019B8BF328
:101410001188E41A1F4486F31188DBE7C1608161FB
:101420004161C3611144009B0060406082600161C2
:1014300003627047F8B504460E461746202383F32F
:101440001188A568A5B1A368013BA36063695A1C14
:1014500062611E70236962699A4224BFE368636116
:10146000E3690BB120469847002080F31188F8BD4E
:101470003946204600F00EFE0028E2DA85F3118896
:10148000F8BD0000836942699A4210B501D18268B3
:101490007AB98268013282605A1C82611C780369C1
:1014A0009A4201D3C3688361002100F003FE204605
:1014B00010BD4FF0FF3010BD2DE9F74F05460F4628
:1014C00090469A46D0F81C90202686F311884FF05B
:1014D000000B144664B1224639462846FFF7EEFE5B
:1014E000034668B95146284600F0D4FD0028F1D0E3
:1014F000002383F31188A8EB040003B0BDE8F08F4C
:10150000B9F1000F03D001902846C847019B8BF327
:101510001188E41A1F4486F31188DBE702684368E8
:101520001143016003B11847704700001430FFF702
:1015300043BF00004FF0FF331430FFF73DBF000002
:101540003830FFF7B9BF00004FF0FF333830FFF7F6
:10155000B3BF00001430FFF709BF00004FF0FF31A8
:101560001430FFF703BF00003830FFF763BF0000FF
:101570004FF0FF323830FFF75DBF000000207047AA
:10158000FFF7D8BD044B0360002343608360C36052
:1015900001230374704700BF703F000810B520237B
:1015A000044683F31188FFF7F3FD0223237400231D
:1015B00083F3118810BD000038B5C36904460D4699
:1015C0001BB904210844FFF7A9FF294604F11400C0
:1015D000FFF7B0FE002806DA201D4FF48061BDE859
:1015E0003840FFF79BBF38BD026843681143016074
:1015F00003B118477047000013B5446BD4F8943416
:101600001A681178042915D1217C022912D119797F
:10161000128901238B4013420CD101A904F14C0023
:1016200001F084FFD4F89444019B2179024620689C
:1016300000F0EAF902B010BD143001F007BF00005D
:101640004FF0FF33143001F001BF00004C3001F0C7
:10165000D9BF00004FF0FF334C3001F0D3BF000082
:10166000143001F0D5BE00004FF0FF31143001F00E
:10167000CFBE00004C3001F0A5BF00004FF0FF329C
:101680004C3001F09FBF0000D0F8942438B51368A7
:1016900019780429054601D0012038BD017C0229B2
:1016A000FAD112795C89012090400440F4D105F10F
:1016B000140001F067FE02460028EDD0D5F89454DE
:1016C0004FF480732868697900F08CF9204638BDA2
:1016D000406BFFF7D9BF0000002070477047000043
:1016E0007FB5124B0360002343608360C360012514
:1016F00002260F4B057404460290019300F1840208
:10170000294600964FF48073143001F017FE094B00
:101710000193029400964FF4807304F523722946D6
:1017200004F14C0001F0DEFE04B070BD983F0008EB
:10173000D1160008F91500080A68202383F31188E0
:101740000B790B3342F823004B79133342F8230013
:101750008B7913B10B3342F8230002230374C0F8D2
:101760009414002383F311887047000038B5037F79
:10177000044613B190F85430ABB9201D0125022165
:10178000FFF732FF04F1140025776FF0010100F03C
:101790009DFC84F8545004F14C006FF00101BDE849
:1017A000384000F093BC38BD10B501210446043028
:1017B000FFF71AFF0023237784F8543010BD000090
:1017C00038B504460025143001F0D0FD04F14C007A
:1017D000257701F09FFE201D84F854500121FFF76A
:1017E00003FF2046BDE83840FFF74EBF90F8803039
:1017F00003F06003202B19D190F88120212A0AD010
:10180000222A4FF000030ED0202A0FD1084A426747
:101810000722826704E0064B4367072383670023A0
:10182000C3670120704743678367F9E7002070476B
:1018300010240020D0F8943437B51A6811780429A0
:1018400004461AD1017C022917D119791289012382
:101850008B40134211D100F14C05284601F01AFFCC
:1018600058B101A9284601F061FED4F89444019BC7
:1018700021790246206800F0C7F803B030BD0000AF
:1018800001F10B03F7B550F8234005460E46F4B1BD
:10189000202383F3118805EB8607201D0821FFF71D
:1018A000A3FEFB685B691B684C3413B1204601F052
:1018B0004BFE01A9204601F039FE024648B1019BCA
:1018C0003146284600F0A0F8002383F3118803B0C6
:1018D000F0BDFB685A691268002AF5D01B8A013BEB
:1018E0001340F1D105F18002EAE70000133138B569
:1018F00050F82140DCB1202383F31188D4F89424DC
:101900001368527903EB8203DB689B695D6845B11C
:1019100004216018FFF768FE294604F1140001F065
:101920003BFD2046FFF7B0FE002383F3118838BD4E
:101930007047000001F036B80123037000234360B4
:1019400000F1300200F1500142F8043B8A42D361B9
:10195000FAD103814381704738B50446202383F3CD
:1019600011880025416000F10C0300F1300243F8BA
:10197000045B9342FBD1204601F036F8022323702A
:1019800085F3118838BD000070B500EB8103054672
:101990005069DA600E46144618B110220021FFF794
:1019A000C1FAA06918B110220021FFF7BBFA314635
:1019B0002846BDE8704001F029B90000038903F012
:1019C00001030381438903F00103438100F13002E5
:1019D00000F11003002143F8041B9342FBD101F0F6
:1019E000ADB90000F0B400EB81044789E46801253B
:1019F000A4698D403D43458123600023A26063605C
:101A0000F0BC01F0C9B90000F0B400EB8104078913
:101A1000E468012564698D403D430581236000230E
:101A2000A2606360F0BC01F041BA0000022310B56F
:101A3000037000230446A0F8883080F88A3080F8CC
:101A40008B300381438100F10C0200F1300142F838
:101A5000043B8A42FBD184F87030204601F06AF8DA
:101A600063681B6823B120460021BDE81040184779
:101A700010BD0000436802781B6880F88C200522A6
:101A800002700BB10421184770470000436890F8BA
:101A90008C201B6802700BB10521184770470000AD
:101AA00090F8703070B5044613B1002380F87030A0
:101AB00004F18002204601F065F963689B6863BB0E
:101AC00094F8805015F0600615D194F8813005F037
:101AD0007F0545EA032540F202339D4200F00E8166
:101AE0005BD8022D00F0DC803FD8002D00F087800D
:101AF000012D00F0CF800021204601F0FBFB0021EA
:101B0000204601F0EBFB63681B6813B106212046F9
:101B10009847062384F8703070BD20469847002807
:101B2000CED094F8872094F8863043EA0223A26F3F
:101B3000934238BFA36794F98030A56F002B4FF014
:101B4000200380F2FD80002D00F0EC80092284F853
:101B5000702083F311880021A36F626F2046FFF786
:101B600053FF002383F3118870BDB5F5817F00F02A
:101B7000B180B5F5407F49D0B5F5807FBBD194F8F1
:101B80008230012BB7D1B4F8883023F00203A4F8D7
:101B900088306667A667E667C3E740F201639D4247
:101BA0001ED8B5F5C06F3BD2B5F5A06FA3D1B4F880
:101BB0008030B3F5A06F0ED194F8823084F88A306B
:101BC000204601F015F863681B6813B10121204617
:101BD00098470323237000236367A367E367A0E7A5
:101BE000B5F5106F32D040F602439D4252D0B5F5A4
:101BF000006F80D104F18B036367012324E004F1BB
:101C0000880363670223A367E5678AE794F8823055
:101C1000012B7FF470AFB4F8883043F00203B6E7CD
:101C200094F88520616894F884304D6894F88310A6
:101C300043EA0223204694F88220A84700283FF474
:101C40005AAF436863670368A367A4E72378042B4C
:101C500010D1202383F311882046FFF7AFFE86F3CF
:101C60001188636884F88B601B68032121700BB1B5
:101C70002046984794F88230002BACD084F88B3003
:101C80000423237063681B68002BA4D00221204624
:101C90009847A0E7374B63670223A36700239DE7BC
:101CA00094F8841011F0800F204601F00F010ED03F
:101CB00001F05AF8012806D002287FF41CAF2E4B01
:101CC0006367A06767E72D4B6367A56763E701F06C
:101CD0003DF8EFE794F88230002B7FF40CAF94F8D6
:101CE000843013F00F013FF476AF1A06204602D578
:101CF00001F018FB6FE701F009FB6CE794F8823004
:101D0000002B7FF4F8AE94F8843013F00F013FF409
:101D100062AF1B06204602D501F0ECFA5BE701F04A
:101D2000DDFA58E7142284F8702083F311882B46DB
:101D30002A4629462046FFF755FE85F3118870BDD7
:101D40005DB1152284F8702083F311880021A36F00
:101D5000626F2046FFF746FE03E70B2284F87020EF
:101D600083F311882B462A4629462046FFF74CFE6E
:101D7000E3E700BFC83F0008C03F0008C43F0008B9
:101D800038B590F870300446152B29D8DFE803F0F9
:101D90003E28282828283E28280B293928282828A2
:101DA000282828283E3E90F8871090F88620836FD8
:101DB00042EA01229A4214D9C268128AB3FBF2F5B0
:101DC00002FB15356DB9202383F311882B462A4673
:101DD0002946FFF719FE85F311880A2384F870302D
:101DE00038BD142384F87030202383F31188002336
:101DF0001A4619462046FFF7F5FD002383F31188A4
:101E000038BDC36F03B198470023E7E7002101F015
:101E100071FA0021204601F061FA63681B6813B172
:101E20000621204698470623D8E7000090F8702046
:101E3000152A38B5044622D80123934040F6416262
:101E400013421DD113F480150FD19B0217D50B231C
:101E500080F87030202383F311882B462A462946C8
:101E6000FFF7D2FD85F3118838BDC3689B695B68B5
:101E70002BB9C36F03B19847002384F8703038BD85
:101E8000002101F037FA0021204601F027FA6368AB
:101E90001B6813B10621204698470623EDE7000092
:101EA000024B00221B605B609A6070471C2E002072
:101EB000002303748268054B1B6899689142FBD22A
:101EC0005A68036042601060586070471C2E002002
:101ED00008B5202383F31188037C032B05D0042B42
:101EE0000DD02BB983F3118808BD436900221A6015
:101EF0004FF0FF334361FFF7DBFF0023F2E790E889
:101F00000C001A6002685360F2E7000000230374BB
:101F10008268054B1B6899689142FBD85A68036038
:101F200042601060586070471C2E0020054B1969F4
:101F30000874186802681A605360186101230374FA
:101F4000FEF742BA1C2E002030B54B1C87B0054668
:101F50000A4C10D023690A4A01A800F0D3F8284699
:101F6000FFF7E4FF049B13B101A800F007F9236910
:101F7000586907B030BDFFF7D9FFF8E71C2E0020E5
:101F8000D11E000838B50C4D41612B6981689A68F3
:101F90009142044603D8BDE83840FFF789BF184690
:101FA000FFF786FF01232C61014623742046BDE81C
:101FB0003840FEF709BA00BF1C2E0020044B1A68F7
:101FC0001B6990689B68984294BF0020012070476D
:101FD0001C2E002010B5084C236820691A68226066
:101FE0005460012223611A74FFF790FF01462069B3
:101FF000BDE81040FEF7E8B91C2E002082600222E6
:1020000002740022427470478368A3F17C0243F893
:102010000C2C026943F83C2C426943F8382C074ADF
:1020200043F81C2CC26843F8102C022203F8082C39
:10203000002203F8072CA3F118007047E103000801
:1020400010B5202383F31188FFF7DEFF002104463B
:10205000FFF798FF002383F31188204610BD00008E
:10206000024B1B6958610F20FFF760BF1C2E002038
:10207000202383F31188FFF7F3BF000008B5014662
:10208000202383F311880820FFF75EFF002383F3EA
:10209000118808BD49B1064B42681B6918605A6037
:1020A000136043600420FFF74FBF4FF0FF307047CD
:1020B0001C2E00200368984206D01A680260506007
:1020C00059611846FFF7F4BE7047000038B5044662
:1020D0000D462068844200D138BD036823605C60EF
:1020E0004561FFF7E5FEF4E7054B03F114025A6181
:1020F0009A614FF0FF32DA6100221A62704700BF26
:102100001C2E0020F8B503611A4BC2605C6A1A4BA2
:102110001A46022952F8145F38BF0221954206463A
:102120001F460AD1586198611C6205604560816054
:102130000819BDE8F84001F0CFBA186AAB68241A54
:102140000C1902D3E41A2D6804E09C4202D2204408
:1021500001F0D2FAAB689C42F4D86B6873603560CA
:102160001E606E60B460A9684FF0FF33091BA96060
:10217000FB61F8BD000C00401C2E002010B41A4C6E
:10218000234653F8141F814210D0416802680A6048
:10219000026851609A424FF00001C16003D0936819
:1021A00081680B4493605DF8044B70470A68626174
:1021B00000209A425360C86003D15DF8044B01F0DF
:1021C00095BA9368886803449360084A206A526A03
:1021D000121A9342E7D9991A012998BF931C1844FF
:1021E0005DF8044B01F088BA1C2E0020000C004062
:1021F00000207047FEE70000704700004FF0FF30FE
:1022000070470000022906D0032906D0012906489C
:1022100018BF0020704705487047032A9ABF04483A
:1022200000EBC20000207047984000084C400008B6
:102230001824002070B59AB001AD0646084629461C
:10224000144600F095F82846FEF764FEC0B2431C21
:102250005B0086E8180023700323637000230234B8
:102260001946DAB2904204F1020401D81AB070BDE6
:10227000EA5C04F8022C04F8011C0133F1E70000C9
:1022800008B5202383F311880348FFF7D3FA00230E
:1022900083F3118808BD00BF5C2E002010B50446F2
:1022A000052916D8DFE801F016150316161D2023A0
:1022B00083F311880E4A0121FFF766FB20460D4A81
:1022C0000221FFF761FB0C48FFF77AFA002383F342
:1022D000118810BD202383F311880748FFF746FAC1
:1022E000F4E7202383F311880348FFF75DFAEDE755
:1022F000CC3F0008F03F00085C2E002038B50C4DA4
:102300000C4C0D492A4604F10800FFF793FF05F134
:10231000CA0204F110000949FFF78CFF05F5CA72E3
:1023200004F118000649BDE83840FFF783BF00BF3D
:1023300024330020182400201C40000824400008FA
:102340003040000870B5044608460D46FEF7E2FD31
:10235000C6B22046013403780BB9184670BD324628
:102360002946FEF7BFFD0028F3D1012070BD000013
:102370002DE9F84F05460C46FEF7CCFD2A49C6B2BA
:102380002846FFF7DFFF08B10136F6B22749284695
:10239000FFF7D8FF08B11036F6B2632E0DD8DFF87C
:1023A0008890DFF888A0224FDFF88CB0DFF88C80AF
:1023B0002E7846B92670BDE8F88F29462046BDE83C
:1023C000F84F01F0B1BD252E29D1072249462846F4
:1023D000FEF788FD40B9D8F800302360D8F8043003
:1023E000636007350834E3E7082251462846FEF7C4
:1023F00079FDA0B90F4BA21C13F8011F09095B4519
:10240000C95D02F8021C197801F00F0102F1020205
:10241000C95D02F8031CEFD118340835C8E72670EF
:1024200001350134C4E700BFB8400008304000085F
:10243000C9400008FFE7F11F0BE8F11FC04000088A
:10244000BFF34F8F044B1A695107FCD1D3F8102109
:102450005207F8D1704700BF0020005208B50D4B5D
:102460001B78ABB9FFF7ECFF0B4BDA68D10741BF24
:102470000A4A5A6002F188325A60D3F80C21D20716
:1024800041BF064AC3F8042102F18832C3F804218F
:1024900008BD00BF8235002000200052230167459F
:1024A00008B5114B1B78F3B9104B1A69510742BF9D
:1024B000DA6842F04002DA60D3F81021520742BFD6
:1024C000D3F80C2142F04002C3F80C21FFF7B8FF0B
:1024D000064BDA6842F00102DA60D3F80C2142F0D0
:1024E0000102C3F80C2108BD8235002000200052F3
:1024F0000F289ABF00F5806040040020704700005C
:102500004FF4003070470000102070470F2808B5C6
:102510000BD8FFF7EDFF00F500330268013204D15C
:1025200004308342F9D1012008BD002008BD00001D
:102530000F2810B504464AD8FFF782FFFFF78EFF39
:1025400024484FF0FF33072C4361C0F8143124D8DE
:102550000361FFF775FF230243F02403C360C368E0
:1025600043F08003C36003695A07FCD4FFF768FF98
:102570002046FFF7BDFF00F50033BFF34F8F164A2B
:10258000984220D3BFF34F8FBFF36F8FFFF788FFC1
:102590002046BDE81040FFF7B9BFC0F81031FFF783
:1025A0004FFFA4F108031B0243F02403C0F80C31D1
:1025B000D0F80C3143F08003C0F80C31D0F8103162
:1025C0005B07FBD4D2E7C2F85C022030D8E70020DA
:1025D00010BD00BF0020005200ED00E02DE9F84FD3
:1025E00042EA0003DB060646884691464AD1FFF7D9
:1025F00035FFDFF8B0B04546A9EB050343441F2B78
:1026000004D8FFF74DFF0120BDE8F88F204A21488C
:10261000214F06F178439342204B214A98BF9A46B6
:1026200003F1FC0386BF1F4692465846FFF708FF9A
:102630004FF0FF3303603B6843F002033B6005F15A
:102640001C022B1FA6EB050EDAF8004014F005045F
:10265000FAD153F8041F4EF803109342F4D1BFF39C
:102660004F8FFFF7EDFE4FF0FF3303603B6823F021
:1026700002033B6020222946304601F045FC20B190
:10268000FFF70EFF0020BDE8F88F20362035B3E7B6
:10269000FFFF0F00142100520C20005210200052A6
:1026A000102100521420005210B5084C237828B194
:1026B00053B9FFF7D3FE0123237010BD23B120705F
:1026C000BDE81040FFF7ECBE10BD00BF8235002012
:1026D00010B50244064B0439D2B2904200D110BD6D
:1026E000441C00B253F8200041F8040FE0B2F4E7B4
:1026F000504000580F4B30B51C6F240405D41C6F9C
:102700001C671C6F44F400441C670B4C236843F4A3
:10271000807323600244094B0439D2B2904200D145
:1027200030BD441C00B251F8045F43F82050E0B2C1
:10273000F4E700BF004402580048025850400058D7
:1027400007B5012201A90020FFF7C2FF019803B0DD
:102750005DF804FB07B502A9012241F8040D002031
:10276000FFF7C8FF03B05DF804FB0000034B1B68D4
:102770005B0142BF024B01221A707047D0440258DD
:1027800083350020014B1878704700BF8335002047
:10279000064A536823F001035360EFF3098368335B
:1027A00083F30988002383F31188704730EF00E03A
:1027B00010B5202383F31188104B5B6813F400637A
:1027C00018D0F1EE103AEFF309844FF0807344F81B
:1027D0004C3C0B4BDB6844F8083CA4F1680383F3E2
:1027E0000988FFF7EBFB18B1064B44F8503C10BDCD
:1027F000054BFAE783F3118810BD00BF00ED00E040
:1028000030EF00E0F1030008F4030008F0B5BFF377
:102810004F8FBFF36F8F1D4B0021C3F85012BFF3D2
:102820004F8FBFF36F8F5A6942F400325A61BFF382
:102830004F8FBFF36F8FC3F88410BFF34F8FD3F860
:102840008020C2F3C904C2F34E325201A50743F6F9
:10285000E07602EA060E284621464EEA00070139D4
:10286000C3F860724F1C00F14040F6D1203A12F1DB
:10287000200FEED1BFF34F8F5A6942F480325A6174
:10288000BFF34F8FBFF36F8FF0BD00BF00ED00E0CF
:10289000FEE70000084A094B09498B4204D3094A64
:1028A0000021934205D3704752F8040F43F8040BFC
:1028B000F3E743F8041BF4E7AC420008503900206A
:1028C0005039002050390020D0F8943030B5002223
:1028D0009D68D0F8904011464FF0FF3004EB421352
:1028E00001329542C3F80019C3F81019C3F808095A
:1028F000C3F8001BC3F8101BC3F8080BEED24FF04F
:102900000113C4F81C3830BD00EB81032DE9F04FF2
:10291000D3F80CE0DEF814404F1CD4F800C03F039D
:102920004FEA41186568D0F8902065450AD3D2F87F
:102930003438012000FA01F123EA0101C2F8341809
:10294000BDE8F08FBEF81060ACEB0503B34228BFC2
:10295000334602EB0806D6F81869B6B2B3EB860F19
:1029600013D8A6683A44A6F1040A99465AF804BF57
:10297000C2F800B0B9F1040F02D9A9F10409F5E7D2
:102980001E442B44A6606360CCE70020BDE8F08FB6
:10299000890141F02001016103699B06FCD41220EA
:1029A00000F03CBF10B50A4C2046FEF7C5FF094BAE
:1029B000C4F89030084BC4F89430084C2046FEF719
:1029C000BBFF074BC4F89030064BC4F8943010BDE1
:1029D0008435002000000840004100082036002017
:1029E000000004400C4100080378012B70B5054637
:1029F0005DD1494BD0F89040984259D1474BD3F81C
:102A0000D82042F00062C3F8D820D3F8002142F069
:102A10000062C3F80021D3F80021D3F8802042F0EF
:102A20000062C3F88020D3F8802022F00062C3F84F
:102A30008020D3F880300E216520FEF7FBFB384B59
:102A4000E360384BC4F800380023C4F8003EC023CC
:102A50002360D5F890604FF40413A3633369002B0F
:102A6000FCDA012333610C2000F0D8FE3369DB0768
:102A7000FCD4122000F0D2FE3369002BFCDA0026D1
:102A8000A6602846FFF720FF6B68C4F81068DB6873
:102A9000C4F81468C4F81C68002B3AD1224BA36117
:102AA0004FF0FF336361A36843F00103A36070BD7F
:102AB0001E4B9842C8D1194BD3F8D82042F000726F
:102AC000C3F8D820D3F8002142F00072C3F80021E7
:102AD000D3F80021D3F8802042F00072C3F88020A0
:102AE000D3F8802022F00072C3F88020D3F8802031
:102AF000D3F8D82022F08062C3F8D820D3F8002180
:102B000022F08062C3F80021D3F800310E214D205D
:102B100093E7074BC3E700BF843500200044025809
:102B20004014004003002002003C30C0203600204A
:102B3000083C30C0F8B5D0F890400546002120464A
:102B4000FFF726FFD5F8941000234FF001128F688D
:102B5000C4F834384FF00066C4F81C284FF0FF303A
:102B600004EB431201339F42C2F80069C2F8006BC4
:102B7000C2F80809C2F8080BF2D20B68D5F8902009
:102B8000C5F89830636210231361166916F01006B9
:102B9000FBD1122000F042FED4F8003823F4FE638B
:102BA000C4F80038A36943F4402343F01003A36141
:102BB0000923C4F81038C4F814380B4BEB604FF0FD
:102BC000C043C4F8103B094BC4F8003BC4F810697B
:102BD000C4F80039D5F8983003F1100243F480139B
:102BE000C5F89820A362F8BDDC40000840800010C2
:102BF000D0F8902090F88A10D2F8003823F4FE63C1
:102C000043EA0113C2F80038704700002DE9F04193
:102C10000EB200EB86080D46D8F80C100F6807F0CE
:102C20000303022B53D0032B53D03F4A3F4F012BBA
:102C300018BF1746D0F890404FEA451E04EB0E032C
:102C40000022C3F8102B8A6905F1100C002A42D02B
:102C50004A8A05F158035B013A43E2500123D4F854
:102C60001C2803FA0CF31343A6444A69C4F81C3821
:102C70000023CEF8103905F13F03002A3BD00A8A21
:102C8000898B9208012988BF4A43D0F8981004EB39
:102C90008303561841EA0242C0F8986029465A60F8
:102CA0002046FFF775FED8F80C301B8A43EA85539F
:102CB0001F4305F148035B01E7500123D4F81C28AA
:102CC00003FA05F51543C4F81C58BDE8F081184F08
:102CD000B0E7184FAEE704EB4613D3F8002B22F40D
:102CE0000042C3F8002BD4F81C28012303FA0CF38C
:102CF00022EA0303B8E704EB83030F4A5A6004EBAC
:102D0000461629462046FFF743FED6F8003923F43D
:102D10000043C6F80039D4F81C38012202FA05F540
:102D200023EA0505CFE700BF0080001000800410F3
:102D30000080081000800C1000040002D0F89420DD
:102D40001268C0F89820FFF7BFBD00005831D0F8D6
:102D5000903049015B5813F4004004D013F4001F75
:102D600014BF0120022070474831D0F8903049014B
:102D70005B5813F4004004D013F4001F14BF01206B
:102D80000220704700EB8101CB68196A0B68136061
:102D90004B6853607047000000EB810330B5DD687D
:102DA000AA691368D36019B9402B84BF402313600C
:102DB0006B8A1468D0F890201C44013CB4FBF3F4F7
:102DC0006343033323F0030302EB411043EAC4439C
:102DD00043F0C043C0F8103B2B6803F00303012B02
:102DE00009B20ED1D2F8083802EB411013F4807FFB
:102DF000D0F8003B14BF43F0805343F00053C0F8B9
:102E0000003B02EB4112D2F8003B43F00443C2F80E
:102E1000003B30BD2DE9F041D0F8906006EB411346
:102E20000546D3F8087BC3F8087B3A070C4608D55B
:102E3000D6F814381B0704D500EB8103DB685B6808
:102E40009847FA072FD5D6F81438DB072BD505EBB2
:102E50008403D968CCB98B69488A5E68B6FBF0F206
:102E600000FB12628AB91868DA6890420DD2121A11
:102E700083E81400202383F3118821462846FFF7B6
:102E80008BFF84F31188BDE8F081012303FA04F27B
:102E90006B8923EA02036B81CB6823B12146284664
:102EA000BDE8F0411847BDE8F081000000EB810368
:102EB00070B5DD68D0F890306C692668E6604A012C
:102EC00056BB1A444FF40020C2F810092A6802F0D9
:102ED0000302012A0AB20ED1D3F8080803EB421408
:102EE00010F4807FD4F8000914BF40F0805040F007
:102EF0000050C4F8000903EB4212D2F8000940F078
:102F00000440C2F80009D3F83408012202FA01F1A2
:102F10000143C3F8341870BD19B9402E84BF402056
:102F2000206020682E8A841940F00050013C1A4429
:102F3000B4FBF6F440EAC440C6E700002DE9F041D6
:102F4000D0F8906006EB41130446D3F80879C3F833
:102F50000879FB070D461CD5D6F81038DA0718D5C6
:102F600000EB8103D3F80CE0DEF81430D3F800C096
:102F7000DA6894451BD2A2EB0C024FF000081A60ED
:102F8000C3F80480202383F31188FFF78FFF88F3B1
:102F900011883B0618D5D6F834280123AB401342DC
:102FA00012D029462046BDE8F041FFF7ADBC012311
:102FB00003FA01F2038923EA02030381DEF80830F1
:102FC000002BE6D09847E4E7BDE8F0812DE9F04713
:102FD000D0F890506E69AB691E40F10404466E61F2
:102FE00003D5BDE8F047FEF721BD002E11DAD5F874
:102FF000003E9A071EBFD5F8003E23F00303C5F834
:10300000003ED5F8043823F00103C5F80438FEF774
:103010003DFD330502D52046FEF72CFDB7040CD547
:10302000D5F8083813F0060FEB6823F470530CBF83
:1030300043F4105343F4A053EB60300704D56368A6
:10304000DB680BB120469847F10200F1A180B20283
:103050000BD5D4F8908000274FF00109D4F89430B4
:103060009B68F9B28B4280F0D280F3061AD5D4F86F
:1030700090100A6AC2F30A1702F00F0302F4F0126A
:10308000B2F5802F00F0EC80B2F5402F0AD104EBAE
:10309000830301F58051DB68186A00231A469F42BA
:1030A00040F0D1803003D5F8185835D5E90303D561
:1030B00000212046FFF7AEFEAA0303D501212046DA
:1030C000FFF7A8FE6B0303D502212046FFF7A2FEFF
:1030D0002F0303D503212046FFF79CFEE80203D50A
:1030E00004212046FFF796FEA90203D505212046BC
:1030F000FFF790FE6A0203D506212046FFF78AFEFD
:103100002B0203D507212046FFF784FEEF0103D5EC
:1031100008212046FFF77EFE700340F1C980E907D1
:1031200003D500212046FFF709FFAA0703D5012197
:103130002046FFF703FF6B0703D502212046FFF768
:10314000FDFE2F0703D503212046FFF7F7FEEE060D
:1031500003D504212046FFF7F1FEA80603D505217B
:103160002046FFF7EBFE690603D506212046FFF750
:10317000E5FE2A0603D507212046FFF7DFFEEB0513
:1031800040F1968020460821BDE8F047FFF7D6BE03
:10319000D4F890904FF000084FF0010AD4F8943022
:1031A0009B685FFA88F7BB42FFF451AF09EB471306
:1031B000D3F8002902F44022B2F5802F24D1D3F8AD
:1031C0000029002A20DAD3F8002942F09042C3F8FF
:1031D0000029D3F80029002AFBDB3946D4F89000F7
:1031E000FFF7D6FB22890AFA07F322EA03032381B9
:1031F00004EB8703DB689B6813B139462046984788
:1032000039462046FFF780FB08F10108C6E708EBC6
:103210004112D2F8003B03F44023B3F5802F10D1C4
:10322000D2F8003B002B0CDA628909FA01F322EA9A
:103230000303638104EB8103DB68DB680BB1204689
:10324000984701370AE713F0030F08BF0A68072BF6
:1032500098BF027003F101039CBF120A01301EE700
:1032600004EB830301F58051DA6890690268D0F8B5
:1032700008C04068A2EB000E00221046974208D119
:10328000DB689B699A683A449A605A6817445F60A1
:1032900008E712F0030F08BF0868964588BF8CF84E
:1032A000000002F1010284BF000A0CF1010CE5E705
:1032B000BDE8F08708B50348FFF788FEBDE8084081
:1032C000FFF776BA8435002008B50348FFF77EFE85
:1032D000BDE80840FFF76CBA20360020D0F89030E7
:1032E00003EB4111D1F8003B43F40013C1F8003B5C
:1032F00070470000D0F8903003EB4111D1F800394D
:1033000043F40013C1F8003970470000D0F8903042
:1033100003EB4111D1F8003B23F40013C1F8003B4B
:1033200070470000D0F8903003EB4111D1F800391C
:1033300023F40013C1F800397047000030B5039C36
:103340000172043304FB0325C361049B0363002162
:10335000059B00604060C16042610261856104625A
:1033600042628162C162436330BD00000022416A53
:1033700041610161C2608262C2626FF00101FEF7C9
:10338000A5BE000003694269934203D1C2680AB135
:1033900000207047181D704703691960C268013228
:1033A000C260C269134482690361934224BF436AC5
:1033B00003610021FEF77EBE38B504460D46E36882
:1033C0003BB16269131D1268A3621344E3620020DB
:1033D00038BD237A33B929462046FEF75BFE002824
:1033E000EDDA38BD6FF00100FBE70000C368C26989
:1033F000013BC3604369134482694361934224BF24
:10340000436A436100238362036B03B1184770472B
:1034100070B52023044683F31188866A3EB9FFF70E
:10342000CBFF054618B186F31188284670BDA36A04
:10343000E26A13F8015BA362934202D32046FFF7CE
:10344000D5FF002383F31188EFE700002DE9F84F43
:1034500004460E4690469946202787F3118800259A
:10346000AA46D4F828B0BBF1000F09D1494620463E
:10347000FFF7A2FF20B18BF311882846BDE8F88F33
:10348000A16AE36AA8EB050B5B1A9B4528BF9B4624
:10349000BBF1400F1BD9334601F1400251F8040B38
:1034A00043F8040B9142F9D1A36A40334036A3623A
:1034B0004035A26AE36A9A4202D32046FFF796FF9C
:1034C0008AF311884545D8D287F31188C9E7304679
:1034D0005A46FDF7FDFCA36A5B445E44A3625D446B
:1034E000E7E7000010B5029C0172043303FB0421DE
:1034F000C36100238362C362039B0363049B006078
:103500004060C4604261026181610462426243635F
:1035100010BD0000026AC260426A4261026100227C
:103520008262C2626FF00101FEF7D0BD4369026999
:103530009A4203D1C2680AB100207047184650F879
:10354000043B0B6070470000C368C2690133C3606D
:103550004369134482694361934224BF436A4361D0
:103560000021FEF7A7BD000038B504460D46E3680C
:103570003BB123691A1DA262E2691344E362002091
:1035800038BD237A33B929462046FEF783FD00284B
:10359000EDDA38BD6FF00100FBE700000369196048
:1035A000C268013AC260C2691344826903619342EE
:1035B00024BF436A036100238362036B03B118478E
:1035C0007047000070B5202304460E4683F311882F
:1035D000856A35B91146FFF7C7FF10B185F3118829
:1035E00070BDA36A1E70A36AE26A01339342A362AC
:1035F00004D3E16920460439FFF7D0FF002080F3AF
:10360000118870BD2DE9F84F04460D4691469A4643
:103610004FF0200888F311880026B346A76A4FB9F7
:1036200051462046FFF7A0FF20B187F311883046AE
:10363000BDE8F88FA06AE76AA9EB06033F1A9F422C
:1036400028BF1F46402F1BD905F1400355F8042B16
:1036500040F8042B9D42F9D1A36A4033A36240365F
:10366000A26AE36A9A4204D3E16920460439FFF76B
:1036700095FF8BF311884E45D9D288F31188CDE799
:1036800029463A46FDF724FCA36A3B443D44A36225
:103690003E44E5E7026943699A4203D1C3681BB916
:1036A000184670470023FBE7836A002BF8D0043BE1
:1036B0009B1AF5D01360C368013BC360C3691A4409
:1036C000836902619A4224BF436A036100238362D3
:1036D0000123E5E700F052B9034B002258631A6159
:1036E0000222DA60704700BF000C0040014B00224C
:1036F000DA607047000C0040014B5863704700BF10
:10370000000C0040FEE7000010B5194CFEF7C8FBA6
:10371000FEF7EAFC802217492046FEF76FFC0123E2
:1037200044F8180C0374144B144AD96821F4E0616E
:103730000904090C0A431249DA60CA6842F080722F
:10374000CA60104A1049C2F8B01F116841F0010167
:1037500011601022DA77202283F82220002383F3DD
:10376000118862B60948BDE81040FEF769BC00BF89
:10377000442E00201841000800ED00E00003FA0587
:10378000F0ED00E0001000E055CEACC5204100088F
:103790002DE9F84F1F4CDFF88090656904F114079C
:1037A0004FF00008D9F82430266AAA689E1B96427A
:1037B0001DD34FF0200AAA68236AD5F80CB0134431
:1037C00023622B68BB425F60A6EB02066361C5F80B
:1037D0000C8001D1FFF78AFF88F311882869D84748
:1037E0008AF311886569AB689E42E4D2DAE76269C0
:1037F000BA420CD0916823628E1B9660A86802289A
:103800002CBF1818981CBDE8F84FFFF775BFBDE82E
:10381000F88F00BF1C2E0020000C0040034B59689D
:103820005A68521A9042FBD8704700BF001000E05F
:103830004B6843608B688360CB68C3600B694361EE
:103840004B6903628B6943620B6803607047000039
:1038500008B52C4B2C48D3F8882040F2FF710A435E
:10386000C3F88820D3F8882022F4FF6222F00702F0
:10387000C3F88820D3F88820D3F8E0200A43C3F89F
:10388000E020D3F808210A43C3F808211F4AD3F8DF
:1038900008311146FFF7CCFF1D4802F11C01FFF76C
:1038A000C7FF1C4802F13801FFF7C2FF1A4802F1B6
:1038B0005401FFF7BDFF194802F17001FFF7B8FF8F
:1038C000174802F18C01FFF7B3FF164802F1A80177
:1038D000FFF7AEFF144802F1C401FFF7A9FF134838
:1038E00002F1E001FFF7A4FF114802F1FC01FFF72C
:1038F0009FFF104802F58C71FFF79AFFBDE8084062
:1039000000F016B900440258000002584041000877
:103910000004025800080258000C02580010025817
:103920000014025800180258001C025800200258C7
:10393000002402580028025808B500F0C7FAFFF723
:10394000E3FEFEF713FFBDE80840FEF7D7BC00001A
:1039500070470000084B1A69920710B508D500247B
:103960001C61202383F31188FFF712FF84F3118871
:10397000BDE81040FEF71CBF000C0040124BD3F80E
:10398000E82042F00802C3F8E820D3F8102142F002
:103990000802C3F810210D4AD3F81031D36B43F05D
:1039A0000803D3630A4B63229A624FF0FF32DA6254
:1039B00000229A615A63DA605A6001225A61082132
:1039C0001A603220FDF736BC004402580010005C3B
:1039D000000C0040F8B5514BD3F880204FF0FF3277
:1039E000C3F880200024D3F88010C3F88040D3F8B7
:1039F0008010D3F88410C3F88420D3F88410C3F85F
:103A00008440D3F88410D96F41F0FF4141F4FF01A5
:103A100041F4DF4141F07F01D967D96F21F0FF41C7
:103A200021F4FF0121F4DF4121F07F01D967D96F33
:103A3000D3F888106FEA41516FEA5151C3F88810EA
:103A4000D3F88810C1F30A01C3F88810D3F888109E
:103A5000D3F89010C3F89020D3F89010C3F890409A
:103A6000D3F89010D3F89410C3F89420D3F894109E
:103A7000C3F89440D3F89410D3F89810C3F8982062
:103A8000D3F89810C3F89840D3F89810D3F88C1056
:103A9000C3F88C20D3F88C10C3F88C40D3F88C106A
:103AA000D3F89C10C3F89C20D3F89C20C3F89C400A
:103AB000D3F89C3000F0EAF9194B07229A60194AB2
:103AC000DA60194A1A6105225A60184A536A43F4A7
:103AD00080335362C2F88440BFF34F8FD2F88030F6
:103AE000C3F3C904C3F34E335B01A50743F6E07685
:103AF00003EA060E284621464EEA00070139C2F8BD
:103B000074724F1C00F14040F6D1203B13F1200F9E
:103B1000EED1BFF34F8FBFF36F8FF8BD0044025853
:103B200090ED00E0000004301B00080300ED00E011
:103B30005A4B5B4901221A605A4B19609A605A4AE3
:103B4000DA6000221A614FF440429A619A69920445
:103B5000FCD51A6842F480721A60544B1A6F12F442
:103B6000407F1FBF4FF480321A6700221A671A681D
:103B700042F001021A604D4A134611684807FCD50D
:103B8000002111611A6912F03802FBD1012119607C
:103B90004FF0804159605A67454ADA62454A1A61D6
:103BA0001A6842F480321A60404A13461168890349
:103BB000FCD5116841F0800111601A68D205FCD56E
:103BC0003D4A3E499A6200225A631963A1F5C02119
:103BD0004B39DA6399635A64394A1A64394ADA62AA
:103BE0001A6842F0A8521A60304B1A6802F0285244
:103BF000B2F1285FF9D109229A610022DA611A62D2
:103C00004FF00052DA643049304A1A6559659A65B6
:103C10002F4A212111601A6942F003021A61234BD5
:103C20001A6902F03802182AFAD1D3F8DC2042F0DF
:103C30000052C3F8DC20D3F8042142F00052C3F84C
:103C40000421D3F80421D3F8DC2042F08042C3F8E9
:103C5000DC20D3F8042142F08042C3F80421D3F8D9
:103C60000421D3F8DC2042F00042C3F8DC20D3F872
:103C7000042142F00042C3F80421D3F80421D3F810
:103C8000F42042F00202C3F8F420D3F81C2142F0E1
:103C90000202C3F81C21D3F81C317047088100517F
:103CA00000C000F000480258020000010044025821
:103CB0000000FF01008890082220400063020701F5
:103CC00047040508FD0BFF010010E0000000011093
:103CD00000200052084A08B5936811680B4003F0B1
:103CE0000103936023B1054A13680BB150689847EC
:103CF000BDE80840FEF75CBD80000058D0380020C9
:103D0000084A08B5936811680B4003F002039360FA
:103D100023B1054A93680BB1D0689847BDE80840C5
:103D2000FEF746BD80000058D0380020084A08B58C
:103D3000936811680B4003F00403936023B1054AB4
:103D400013690BB150699847BDE80840FEF730BDD4
:103D500080000058D0380020084A08B593681168E0
:103D60000B4003F00803936023B1054A93690BB13C
:103D7000D0699847BDE80840FEF71ABD800000589A
:103D8000D0380020084A08B5936811680B4003F04A
:103D90001003936023B1054A136A0BB1506A984728
:103DA000BDE80840FEF704BD80000058D038002070
:103DB000174B10B59C681A68144004F478729A6026
:103DC000A30604D5134A936A0BB1D06A98476006DC
:103DD00004D5104A136B0BB1506B9847210604D5DC
:103DE0000C4A936B0BB1D06B9847E20504D5094A96
:103DF000136C0BB1506C9847A30504D5054A936C1E
:103E00000BB1D06C9847BDE81040FEF7D1BC00BFA5
:103E100080000058D03800201A4B10B59C681A68F2
:103E2000144004F47C429A60620504D5164A136D6E
:103E30000BB1506D9847230504D5134A936D0BB110
:103E4000D06D9847E00404D50F4A136E0BB1506E45
:103E50009847A10404D50C4A936E0BB1D06E9847D5
:103E6000620404D5084A136F0BB1506F98472304BE
:103E700004D5054A936F0BB1D06F9847BDE8104049
:103E8000FEF796BC80000058D0380020062108B507
:103E90000846FDF7CFF906210720FDF7CBF90621EB
:103EA0000820FDF7C7F906210920FDF7C3F906210F
:103EB0000A20FDF7BFF906211720FDF7BBF90621FF
:103EC0002820BDE80840FDF7B5B9000008B5FFF7A8
:103ED00081FD00F00DF8FDF753FBFDF72BFDFDF71D
:103EE000FDFBFFF735FDBDE80840FFF7F3BB000021
:103EF000002304491A465A50C8180833802B4260E0
:103F0000F9D17047D038002010B5013902449042F1
:103F100001D1002010BD10F8013B11F8014FA34260
:103F2000F5D0181B10BD0000034611F8012B03F853
:103F3000012B002AF9D17047121012131211000040
:103F40005C2E0020B029002053544D333248373FB7
:103F50003F3F3F3F000000000096000000000000CF
:103F60000000000000000000000000000000000051
:103F700000000000491500083515000871150008FB
:103F80005D15000869150008551500084115000861
:103F90002D1500087D1500080000000055160008CA
:103FA000411600087D1600086916000875160008FD
:103FB000611600084D16000839160008D9160008C9
:103FC00000000000010000000000000002000000EE
:103FD0000000000081180008ED18000840004000B3
:103FE000F432002004330020020000000000000032
:103FF000030000000000000031190008000000006C
:104000001000000014330020000000000100000038
:10401000000000008435002001010200486F6C7927
:1040200062726F00447572616E64616C2D424C0067
:104030002553455249414C25000000009D220008AF
:1040400005220008ED170008812200084300000047
:104050005440000809024300020100C03209040074
:1040600000010202010005240010010524010001E5
:10407000042402020524060001070582030800FF4C
:1040800009040100020A00000007050102400000C7
:10409000070581024000000012000000A040000857
:1040A000120110010200004062314B0000020102C7
:1040B000030100000403090425424F415244250036
:1040C000447572616E64616C003031323334353660
:1040D00037383941424344454600000000000000A3
:1040E000A11A0008811D00082D1E00084000400094
:1040F000BC360020BC36002001000000CC36002079
:1041000080000000400100000800000000010000E5
:1041100000040000080000006D61696E00000000EE
:1041200038410008D8360020D038002001000000B7
:10413000053700080000000069646C65000000009D
:104140000000802A00000000AAAAAAAA000000001D
:10415000FFFF00000000000000A00A0004000000B3
:1041600000000000AAAAAAAA00000000FDFF0000AB
:1041700000000000000000000050000000000000EF
:10418000AAAAAAAA000000003FFF00000000000049
:10419000000000000000000000000000AAAAAAAA77
:1041A00000000000FFFF0000000000000000000011
:1041B0000000020000000000AAAAAAAA0000010054
:1041C000FFFF0000000000000700000000200000CA
:1041D00000000000AAAAAAAA00100000FFFF000029
:1041E00000000007000000000000000000000000C8
:1041F000AAAAAAAA00000000FFFF00000000000019
:10420000000000000000000000000000AAAAAAAA06
:1042100000000000FFFF00000000000000000000A0
:104220000000000000000000AAAAAAAA00000000E6
:10423000FFFF000000000000000000000000000080
:1042400000000000AAAAAAAA00000000FFFF0000C8
:10425000000000000000000000000000000000005E
:10426000AAAAAAAA00000000FFFF000000000000A8
:104270000000000000000000FF000000000000003F
:10428000483F00083F0000000096000000000800C2
:1042900004000000B440000800000000000000001E
:1042A000000000000000000000000000000000000E
:00000001FF
